:10E000008E00FFBDE54DCE0000DFD0DFD7DFD58627
:10E010005397D9CEE4EBBDE3F8CEE506BDE3F8BDFA
:10E02000E44BCE00C0BDE492BDE49C4D27EB81449F
:10E0300026037EE059814726037EE175815326033E
:10E040007EE18E814C26037EE1F6815026037EE23E
:10E05000E7CEE523BDE3F820C008BDE492BDE4A708
:10E060005D2615BDE492A60026E796D18B8097D356
:10E0700096D0890097D2203896DB97D196DA97D040
:10E08000BDE492A600812C27114D26C596D18B8028
:10E0900097D396D0890097D2201608BDE492BDE4AC
:10E0A000A7BDE4925D27AA6D0026A6DEDA08DFD2BE
:10E0B00096D184F097DD96D097DC7F00D48D21BD7A
:10E0C000E565261196D4810225F396D397D196D291
:10E0D00097D07EE01996DD97D196DC97D07EE01937
:10E0E00096DCD6DDBDE403CEE52BBDE3F8CE00C063
:10E0F000DFDEC6108D295A26FBCEE52EBDE3F8CE15
:10E1000000C0C610A6000881202509817F2405BD16
:10E11000E56B2005862EBDE56B5A26E87EE4418638
:10E1200020BDE56B96D4262596D091DC260696D1A7
:10E1300091DD27158620BDE56BBDE56BDEDEA70012
:10E1400008DFDEDEDC08DFDC39860197D496D48177
:10E150000126E1DEDCA60008DFDCDEDEA70008DF4A
:10E16000DEBDE40696D291DC260A96D391DD260424
:10E17000860297D43908BDE492BDE4A7A600270320
:10E180007EE0515D2704DEDADFD5DED56E0008BD06
:10E19000E492BDE4A7BDE4926D0026575D2702DE40
:10E1A000DADFD796D7D6D8BDE403CEE52EBDE3F8A7
:10E1B000DED7A600BDE4068620BDE56BBDE44BCEF0
:10E1C00000C0BDE492A6002607DED708DFD720D125
:10E1D000812D2607DED709DFD720C6812E26037EB4
:10E1E000E019BDE4A75D270BDED796DBA70008DFAB
:10E1F000D720AE7EE05108BDE492BDE4A7BDE49215
:10E200006D0026EFBDE55ABDE49C8153276F813A2E
:10E21000270D810D27EE810A27EABDE55A20F3BDBF
:10E22000E41B97E016BDE41B97DC9BE097E0BDE4A0
:10E230001B97DD9BE097E096DD9BDB97DD96DC99F5
:10E24000DA97DCDEDCBDE41B97E19BE097E05D271D
:10E2500014BDE41B369BE097E0327D00E12603A766
:10E2600000085A26ECBDE41B9BE026087D00E12750
:10E27000A97EE019CEE509BDE3F87EE019BDE55AB7
:10E2800097E1BDE41B1697E0BDE41B97DC9BE0978C
:10E29000E0BDE41B97DD9BE097E096DD9BDB97DD1F
:10E2A00096DC99DA97DCDEDCC0032718BDE41B3668
:10E2B0009BE097E096E18131260632A70008200115
:10E2C000325A26E8BDE41B9BE081FF261196E181CE
:10E2D0003727118138270D813927097EE21ACEE5CB
:10E2E00016BDE3F87EE01908A600BDE49C8149272D
:10E2F00004815326030897D9BDE492BDE4A75D27A6
:10E300002296DA97DE96DB97DFBDE492A600812C99
:10E31000261108BDE492BDE4A75D2707BDE4926D18
:10E320000027037EE051DEDA08DFDA96DB90DF9724
:10E33000DB96DA92DE97DADEDE8D1E96DA9ADB263F
:10E34000F896D981492609CEE532BDE3F87EE01979
:10E35000CEE540BDE3F87EE019C6107D00DA260662
:10E3600096DB1124011696DB1097DB96DA82009774
:10E37000DA96D98149263F863ABDE56B17BDE4069A
:10E38000D7E0DFDE96DEBDE40696DE9BE097E09602
:10E39000DFBDE40696DF9BE097E04FBDE406A600F4
:10E3A00036BDE406329BE097E0085A26F196E0403D
:10E3B000BDE4067EE4418653BDE56B8631BDE56B69
:10E3C000178B0397E0BDE406DFDE96DEBDE406961C
:10E3D000DE9BE097E096DFBDE40696DF9BE097E0EA
:10E3E000A60036BDE406329BE097E0085A26F19677
:10E3F000E043BDE4067EE441A6002706BDE56B08C8
:10E4000020F6398D011736444444448D0132840F7F
:10E410008B30813A25028B077EE56B4F8D0448488F
:10E4200048483716BDE55ABDE49C81302511813A34
:10E43000250A8141250981472405800780301B3347
:10E4400039860DBDE56B860A7EE56BCE00C05FBDEB
:10E45000E55A810D2737810A273381082719817FE3
:10E460002715812025E9818024E5C10F24E15CA7DF
:10E470000008BDE56B20D85D27D55A098608BDE5A3
:10E480006B8620BDE56B8608BDE56B20C28DB26F43
:10E490000039A600812026030820F739816125066E
:10E4A000817B24028BE0395F7F00DA7F00DBA600EE
:10E4B0008DEA81302534813A250A8141252C814716
:10E4C00024288007803049494949497900DB79008F
:10E4D000DA497900DB7900DA497900DB7900DA4939
:10E4E0007900DB7900DA085C20C4390D0A556E69C1
:10E4F00076657273616C204D6F6E69746F72203631
:10E500003830300D0A005D20004572726F7220694C
:10E510006865780D0A004572726F722073726563C8
:10E520000D0A004572726F720D0A00203A00203AFF
:10E5300020003A303030303030303146460D0A005D
:10E54000533930333030303046430D0A008603B73C
:10E55000801801018615B7801839B6801884012704
:10E56000F9B6801939B6801884013936B680188416
:08E570000227F932B7801939C6
:08FFF800000000000000E00021
:00000001FF
